:100000000C9434000C9451000C9451000C94510049
:100010000C9451000C9451000C9451000C9451001C
:100020000C9451000C9451000C9451000C9451000C
:100030000C9451000C9430010C9451000C9451001C
:100040000C9451000C9451000C9451000C945100EC
:100050000C9451000C9451000C9451000C945100DC
:100060000C9451000C94510011241FBECFEFD4E02A
:10007000DEBFCDBF11E0A0E0B1E0ECEAF2E002C0EB
:1000800005900D92A032B107D9F711E0A0E2B1E0DE
:1000900001C01D92A032B107E1F70E94C2000C948A
:1000A00054010C940000569A20E030E05F9890E0F4
:1000B00080FF02C05E9A01C05E985F9A2F5F3F4F3B
:1000C0002830310519F095958795F0CF0895569809
:1000D00040E020E030E061E070E05F985F9A4E9B86
:1000E00008C0CB01022E02C0880F991F0A94E2F7C4
:1000F000482B2F5F3F4F2830310579F7842F089523
:100100001F93162F5F985D9A90E08F719070880F03
:10011000991F80680E945300812F0E9453005D98B0
:100120001F9108955F985D9A90E08F719070880F8D
:10013000991F81680E9453000E9467005D9808958E
:10014000389A399A3A9A3B9A3C9A3D9A559A569AD5
:10015000579A4098439A459A87E060E00E94800051
:1001600080E060E00E94800081E060E00E9480000A
:100170001092800082E08093810081E080936F0084
:10018000789408950E94A00083B7816083BF88950A
:1001900083B78E7F83BFF8CF20E030E0482F50E058
:1001A0004498CA01022E02C0959587950A94E2F7F9
:1001B00080FF02C0409801C0409A449A2F5F3F4F91
:1001C0002830310569F70895CF92DF92EF92FF92C0
:1001D0000F931F9380E00E949200C82EDD2481E0DF
:1001E0000E949200082F10E04298F80134E0F69542
:1001F000E7953A95E1F720E0E22E21E0F22EEE0FAE
:10020000FF1FEE0DFF1D80810E94CC000F7010704B
:10021000000F111F0E0D1F1DF80180810E94CC00E0
:10022000F601B4E0F695E795BA95E1F7EE0FFF1FFA
:10023000EE0DFF1D80810E94CC00FFE0CF22DD2467
:10024000CC0CDD1CEC0CFD1CF70180810E94CC0065
:10025000429A1F910F91FF90EF90DF90CF900895F9
:100260001F920F920FB60F9211242F933F934F932B
:100270005F936F937F938F939F93AF93BF93EF930E
:10028000FF930E94E400FF91EF91BF91AF919F9186
:100290008F917F916F915F914F913F912F910F902F
:0C02A0000FBE0F901F901895F894FFCF30
:1002AC007B006000570076006C003E003F00700041
:1002BC007F007C007D002F00070067001F001D00E1
:00000001FF
